:020000040000FA
:020000001728BF
:08000800C000030EC1000B1B38
:100010000C1C0D2864200C1012288B1A0B1D1228A2
:1000200065200B11410E8300C00E400E090083169F
:10003000FF2390008312203084008001840A041F73
:100040001D28841E1D288316810196018C019901AB
:1000500083120730990090018316850195018B0169
:100060008B170B178C018101011481140115831268
:10007000143085000030A4005D20A600A1000E30E1
:10008000A3008B162008031942282008031D4528C9
:100090000030A4002608A5004E204228831624081C
:1000A0009B0025089A001C158B1355309D00AA3023
:1000B0009D009C148B1783120800831624089B0054
:1000C0001C141A08831208000800A30B9B28073091
:1000D000A300A00AA10B9B282608A2000301260763
:1000E000A20B6F28A607A60A260C1F39A200A2079A
:1000F000A207A207A207A20CA20CA20CA20CA20C9F
:100100000730A205031D8728013085069828A20B19
:100110008C28023085069828A20B91280430850689
:100120009828A20B9628103085069828203085063E
:080130002608A10000000800F0
:02400E00843FED
:00000001FF
